:020000040000fa
:080000001406040000000000da
:020000040000fa
:020000040002f8
:04afe000dfff00008f
:020000040000fa
:020000040002f8
:04afe400ffff00006b
:020000040000fa
:020000040002f8
:04afe80078ff0000ee
:020000040000fa
:020000040002f8
:04afec007dff0000e5
:020000040000fa
:020000040002f8
:04aff00078ff0000e6
:020000040000fa
:1000080000000000000000000000000000000000e8
:100018000c060000000000000000000000000000c6
:10002800000000000000000000000000b00900000f
:1000380000000000000000000000000000000000b8
:10004800f20900000000000000000000bc0a0000e7
:10005800280b0000540b0000000000000000000006
:100068000000000000000000000000000000000088
:100078000000000000000000000000000000000078
:10008800000000000000000000000000380a000026
:100098007a0a0000000000000000000000000000d4
:1000a8000000000000000000000000000000000048
:1000b8000000000000000000000000000000000038
:1000c8000000000000000000000000000000000028
:1000d8000000000000000000000000000000000018
:1000e8000000000000000000000000000000000008
:1000f80000000000000000000000000000000000f8
:1001080000000000000000000000000000000000e7
:1001180000000000000000000000000000000000d7
:1001280000000000f40a00000000000000000000c9
:1001380000000000000000000000000000000000b7
:1001480000000000000000000000000000000000a7
:100158000000000000000000000000000000000097
:100168000000000000000000000000000000000087
:100178000000000000000000000000000000000077
:100188000000000000000000000000000000000067
:100198000000000000000000800b0000ac0b000015
:1001a800d80b000000000000000000000000000064
:1001b8000000000000000000000000000000000037
:1001c8000000000000000000000000000000000027
:1001d8000000000000000000000000000000000017
:1001e8000000000000000000000000000000000007
:1001f80000000000000000000000000000000000f7
:1002080000000000000000000000000000000000e6
:1002180000000000000000000000000000000000d6
:1002280000000000000000000000000000000000c6
:1002380000000000000000000000000000000000b6
:1002480000000000000000000000000000000000a6
:100258000000000000000000000000000000000096
:100268000000000000000000000000000000000086
:0c0278000000000000000000000000007a
:020000040000fa
:1004000027d2bf002652b7004220af002672ec0070
:1004100027d2d60027d2b60000c0d20027d2bf0014
:1004200000c0fd0027f2b70026d2bf0000c0fd00cb
:100430000040d20027d2b60027d2bf0000c0fd0086
:1004400027f2b7001040b20026f2d60026f2b6001e
:1004500027f2d6003091800000000600803e200088
:10046000030007008100e900fcff3a0000000600dd
:10047000831f7800c20320000400bc006601510005
:10048000e0815900f23fb1000380b1000600350061
:10049000ee03090000000000423fb1000380b100fc
:1004a000fbff3d001200b000223fb000020035000b
:1004b0000280090000000000cf0178000000060063
:1004c000889fbe008a9fbe008c1f78000004be007b
:1004d000850107000478a30026003a006120e100ae
:1004e0002500320009f8a30025003a006420e1004d
:1004f00021003200f507b1000508a3000200320018
:1005000000004000818048006044b80003102000d3
:1005100002002000000040008180480008054400df
:1005200089854c000a0541008b8549000a05500069
:100530008b855800030033000a00be0002047400db
:10054000838474008301d1000281d300830f710082
:10055000f0ff3a008904d1000884d300600149000b
:1005600082017800c1adde00fb07b0007301070017
:10057000070037000960a0000800be000400370033
:100580001202200062918800f0ff2f00f1ff270087
:100590004f0678004f05be004f04be000000060065
:1005a00003f0a200869fbe00889fbe008a9fbe0007
:1005b0008c9fbe0044010700860133006450e100b7
:1005c0004f0032006420e1005200320003826c00d0
:1005d00007003b000905d0000306d000820f54003d
:1005e0000c065d000200390002003200890178002b
:1005f000030678008582550004003d000003fd00dd
:100600008103fd008502ea008b854200840f7200a1
:1006100002003b0060001000e08018006011b8008c
:100620000005eb007a28e1000a0039000600780096
:10063000c75ddd00f707b200878075002d00370029
:10064000828171000a017800610560008180d1001b
:100650000080d3008502e900f9ff3b00060440005a
:100660008784480002003b0060041400e0841c0002
:100670000988a300070032008a817100828171001d
:10068000610164008904d1000884d3008b05e8006f
:10069000170037000978a30013003a000b00e000b0
:1006a000130034008b05e9000804440089844c00e1
:1006b0000a4474000978a3000d003a000b00e00022
:1006c000070034008b05e9000804440089844c00cd
:1006d00001003a000b0020000978a300f7ff320068
:1006e0000001eb0002003700828171000a017800ee
:1006f000120107000cf0a70001f0a0003e01370036
:100700006420e10002003a00838f6c003f01330057
:100710000801be000200be0037013700869fbe0000
:10072000889fbe008a9fbe008c9fbe00e600070027
:100730002801330003866c006450e1002e00320073
:100740006420e100330032006150e1002f003200ec
:100750006120e1003100320085855500eb07b000d3
:1007600009002000080420000500370008044400a8
:1007700089844c000a0031000603430087834b0044
:100780000001530081815b00f8ff33000203be00cb
:100790000800a0000804440089844c00f6ff3900da
:1007a000c639dd0083017300010032001300200010
:1007b0008904d1000884d3000998a3000500320001
:1007c0000800a7000300a0008904d1000884d3001a
:1007d0008b05e8008904d1000884d3000001eb00f8
:1007e0000281d200d500070001f0a1000cf0a700a3
:1007f00001f0a000000137006420e1000301320095
:100800000801be000200be00f7ff37006120e100d2
:10081000fe0032006000b800f3ff37000000200047
:1008200001f82700f0ff3700869fbe00889fbe00ba
:100830008a9fbe008c9fbe00a3000700e500330026
:1008400003866c006450e100240032006420e10063
:10085000270032006150e100220032006120e100f7
:10086000210032008b854200eb07b1000134b80053
:10087000003ab8000804420089844a00013ab800ee
:100880000030b8008880400009014a0004003300ad
:100890000000400081804800020149008b05e9000a
:1008a000c909dd008301700001003200130020003f
:1008b000c814de004814dd004709de001200b20053
:1008c000c808de00088470009c00070001f0a10049
:1008d0000cf0a70001f0a000c70037006120e10084
:1008e000ca0032000801be000200be00f7ff370058
:1008f0006150e100fcff3a00c4003700829fbe0057
:100900000001be00780007000470a70003f0a100fa
:100910006509b100180032000e0035006828e100ba
:1009200007003500f0ff2f00f1ff27000300e00073
:1009300015003b00010028004f01be00000005002b
:1009400000004000818048008502e900fcff3a0079
:1009500009003700f88f420003003c008000eb00e4
:100960004f01be00000005008100d1000080d300cf
:100970008502e800fcff3a000300e00002003b00b3
:1009800060001000e08018004f01be00000006006b
:10099000829fbe000001be00530007000470a70044
:1009a00003f0a10003f8a30015003a006509b100a7
:1009b000110032000a0035006928e100030035000b
:1009c000010028004f01be000000050000004000ab
:1009d000818048008502e900fcff3a0006003700ec
:1009e000f88f4200060035008100d1000080d3005e
:1009f0008502e800fcff3a004f01be00000006003f
:100a00008000eb004f01be00000005000080fb00ed
:100a10008000eb00829fbe00889fbe008a9fbe00c0
:100a2000010578000100e0000400350008003c00ea
:100a30000000e000200032000500370060001000d8
:100a4000e080180002003b0001f024001a0037008b
:100a50000004be006011b8006b0920000982cf00bd
:100a6000020039000882cf000441b0006942520000
:100a70000e00320008003b008281710061016400b9
:100a80008904d1000884d3008b05e8000442e80003
:100a9000f9ff3a00050037000804440089844c003f
:100aa0008b05e9000442e900fbff3a002300070040
:100ab0000af0a70001f0a0004f05be004f04be00e1
:100ac0004f01be00000006000004be000600070043
:100ad0000003be000405be000200be0002000700c5
:100ae000844f750000000600c70ade00f107b2005f
:100af000f50fb20008003200e1cf420002003200e0
:100b00000170a00024000500810f70000100320078
:100b10000408050044000500810f700002003a003f
:100b2000140005008502e9000000400081c0480073
:100b3000fcff3b000170a0002400050081002000a4
:100b4000618055000b003d000b00200061fe2f006e
:100b50000100e1001d003400828171006101640028
:100b60008904d1000884d3000000e800faff3a00ad
:100b7000710020006100640003007000020060004a
:100b80000900320061044400e0844c000988a5009b
:100b9000050032008b05e8006808e10002003a0019
:100ba0008904d1000884d300f20f20000258e1002c
:100bb00005003d00c75ddd00f907b20089807500c2
:100bc00008007800000006000bf827008b00780072
:100bd000000005000200be006450e1000500360080
:100be0006420e100020036000968a30001003a0019
:100bf0000800be000160a0004f06be004f05be0009
:100c00004f04be004f03be0000000600f0ff2f009f
:100c1000f1ff2700f8ff37000020ef000220ef006f
:100c2000c088a900004006000f002100b02e21005e
:100c300000018800000000000000eb0000077800c1
:100c40000c000900002f78000007eb005420ef0093
:100c50000e2eef001e2eef000000eb00a121210060
:100c6000e51d09008018780010cea90010cea9005b
:100c700014cea90010aea90010aea90014aea900b0
:100c8000108ea90040a7a900a1002000f3fd0700d5
:100c9000e0022000303a880044e7a90044c7a900d8
:100ca0004407a9004427a9004447a9004467a900b4
:100cb0004487a900300020000600fc0031742000a9
:100cc00082072000a309200082487800834878002a
:100cd00080487800113a8000618070000600fc00b6
:100ce00021742000620420007305200082487800ef
:100cf00083487800804878004427ef00e002200015
:100d0000303a8800300020000d00fc0031742000d3
:100d100082072000a30920008248780083487800d9
:100d20008048780000002000217420006204200028
:100d30007305200082487800834878008048780056
:100d400042a7ae00feff3700813e2000c3fd070032
:100d500010c0b30086e6b70090c2b300c4e6b70087
:100d6000000220000070880000702500807088005c
:100d700010eea9004188a80041a8a80041c8a90018
:100d800004a1a9000481a90005e1a8000068a90048
:100d90001061a8001021a90011e1a80011a1a9006b
:100da00010a1a8001081a8000821ef000621ef0083
:100db0000ca1ef000ea1ef004408a8004428a900f0
:100dc0004448a9000108a9002108a8001fe1a800c3
:100dd0001fa1a9001ec1a9001ea1a9001e81a90072
:100de0001e61a9001e21a9004d88a9004da8a800d8
:100df0004dc8a8000368a90021e1a80021a1a9000d
:100e000020c1a90020a1a9002081a9002021a900ba
:100e10004e08a9004e28a8004e48a8000388a90043
:100e20002002a9002022a9002042a90020a2a90096
:100e30002062a9002082a90020e2a9002102a900c5
:100e40002122a900700720004011880022a2a900d9
:100e500022c2a90022e2a90021e2a8002182a90061
:100e60004588a90045a8a80045c8a8002168a80091
:100e70002828a80023e2a90023e2a9002342a80011
:100e80002362a9000188a9002188a8004608a800bb
:100e90004628a8004648a9002bc8a9002be8a900ad
:100ea0002c08a9000bc8a9000be8a9000c08a90090
:100eb00001eca90001aca900016ca900014ca9003a
:100ec000012ca900010ca90000eca900008ca900cc
:100ed00000aca90000cca900000ca900002ca900be
:100ee000004ca900006ca900202cef00402cef0062
:100ef000602cef00f01f200020608800020ca90089
:100f0000022ca900024ca900262cef00462cef0071
:100f1000662cef00282cef00482cef00682cef0027
:100f20000aacef0023eca80023cca90043eca800f6
:100f300043cca90063eca80063cca900dabc2a006a
:100f40001b32240030002c00fa608800fb6088000f
:100f500020618800dabc2a001b322400000028002f
:100f6000fa608800fb60880010618800dabc2a0003
:100f70001b32240030002c00fa608800fb608800df
:100f800020628800dabc2a001b32240000002800fe
:100f9000fa608800fb60880010628800dabc2a00d2
:100fa0001b32240030002c00fa608800fb608800af
:100fb00020638800dabc2a001b32240000002800cd
:100fc000fa608800fb6088001063880011eea900b9
:100fd00011aea900116ea900a70037003f0037002d
:100fe00000202000006188000020200000628800ae
:100ff0000020200000638800020ca900022ca80039
:10100000024ca80004acef0028acef0048acef00a5
:1010100068acef00262cef00462cef00662cef00aa
:101020000aacef0023eca80023cca90043eca800f5
:1010300043cca90063eca80063cca900dabc2a0069
:101040001b32240030002c00fa608800fb6088000e
:1010500020618800dabc2a001b322400000028002e
:10106000fa608800fb60880010618800dabc2a0002
:101070001b32240030002c00fa608800fb608800de
:1010800020628800dabc2a001b32240000002800fd
:10109000fa608800fb60880010628800dabc2a00d1
:1010a0001b32240030002c00fa608800fb608800ae
:1010b00020638800dabc2a001b32240000002800cc
:1010c000fa608800fb6088001063880011eea900b8
:1010d00011aea900116ea900670037003500370076
:1010e00000102000006188000010200000628800cd
:1010f0000010200000638800020ca900022ca80048
:10110000024ca8000a2cef0004acef00282cef00e2
:101110005055250040628800a0aa2a00406388003c
:10112000dabc2a001b32240030002c00fa60880050
:10113000fb60880020618800dabc2a001b32240092
:1011400000002c00fa608800fb60880010618800b5
:10115000dabc2a001b32240030002c00fa60880020
:10116000fb60880020628800dabc2a001b32240061
:1011700000002c00fa608800fb6088001062880084
:10118000dabc2a001b32240030002c00fa608800f0
:10119000fb60880020638800dabc2a001b32240030
:1011a00000002c00fa608800fb6088001063880053
:1011b0003100370030003700001020000061880047
:1011c0000010200000628800020ca900022ca80078
:1011d000024ca8000a2cef0004acef00282cef0012
:1011e0000000240040628800dabc2a001b32240080
:1011f00030002c00fa608800fb60880020618800c5
:10120000dabc2a001b32240000002c00fa6088009f
:10121000fb60880010618800dabc2a001b322400c1
:1012200030002c00fa608800fb6088002062880093
:10123000dabc2a001b32240000002c00fa6088006f
:10124000fb60880010628800dabc2a001b32240090
:1012500030002c00fa608800fb6088002063880062
:10126000dabc2a001b32240000002c00fa6088003f
:10127000fb60880010638800218ca900418ca900c4
:10128000618ca900216ca900416ca900616ca900c6
:10129000214ca900414ca900614ca90020eca800f8
:1012a00040eca80060eca8003e2cef005e2cef00a4
:1012b0007e2cef0001eca8000000eb00414e210065
:1012c000ff00090080587800bf72ef00c072ef0085
:1012d000a232ef00a432ef000000eb00415e2100db
:1012e0000801090080587800c172ef00c272ef0057
:1012f0000080eb00814d2100050009008018780076
:101300004832ef004a32ef004c32ef00d472ef0067
:101310002e0b0700f60a0700450b07005032ef00be
:10132000a0a48000e0908800b0a480001c12b5004a
:10133000e0908800b0a4800010918800c0a48000d4
:101340002212b5001c12b4004200de007092880028
:101350005232ef005432ef005632ef0037013700bf
:10136000ff3ffc004200f8003600f8004400f8009f
:101370008e1f78000e0020000d000900be1f7800af
:101380003200f8000100fc000068a9000021ef0015
:1013900013eeaf000400370090948000100888001e
:1013a00015eea80004003700009580009412b500e7
:1013b0001008880015eea900ff3ffc003200f9007c
:1013c000ae0120000d0009004f1778004f0778008c
:1013d0004400f9003600f9004200f9000100fc0069
:1013e00000400600ff3ffc004200f8003600f80015
:1013f0004400f8008e1f78000e0020000d00090048
:10140000be1f78003200f8000100fc000108a900ae
:101410000821ef000621ef000080eb00814d210044
:101420000500090080187800d2f2ef00a232ef0028
:10143000a432ef00a5f2a900d572ef00d672ef003a
:10144000d772ef00ff3ffc003200f900ae01200030
:101450000d0009004f1778004f0778004400f9008d
:101460003600f9004200f9000100fc0000400600cf
:10147000ff3ffc004200f8003600f8004400f8008e
:101480008e1f78000e0020000d000900be1f78009e
:101490003200f8000100fc000368a9001421ef00ed
:1014a00013aeaf0004003700b0948000d00888006d
:1014b00015aea80004003700009580009812b50012
:1014c000d008880015aea900ff3ffc003200f900eb
:1014d000ae0120000d0009004f1778004f0778007b
:1014e0004400f9003600f9004200f9000100fc0058
:1014f00000400600ff3ffc004200f8003600f80004
:101500004400f8008e1f78000e0020000d00090036
:10151000be1f78003200f8000100fc000388a9001b
:101520001821ef00136eaf0004003700d094800044
:10153000e0088800156ea8000400370000958000c0
:101540009c12b500e0088800156ea900ff3ffc0062
:101550003200f900ae0120000d0009004f1778009d
:101560004f0778004400f9003600f9004200f90006
:101570000100fc0000400600ff3ffc004200f800b4
:101580003600f8004400f8008e1f78000e0020009e
:101590000d000900be1f78003200f8000100fc00b9
:1015a0000168a900bf72ec00bfd2bf008080fb00c1
:1015b00030118000424e210080707900ff3ffc0016
:1015c0003200f900ae0120000d0009004f1778002d
:1015d0004f0778004400f9003600f9004200f90096
:1015e0000100fc0000400600ff3ffc004200f80044
:1015f0003600f8004400f8008e1f78000e0020002e
:101600000d000900be1f78003200f8000100fc0048
:101610000828a9002242ae00000037002222af00b5
:101620002222a900ff3ffc003200f900ae01200099
:101630000d0009004f1778004f0778004400f900ab
:101640003600f9004200f9000100fc0000400600ed
:10165000ff3ffc004200f8003600f8004400f800ac
:101660008e1f78000e0020000d000900be1f7800bc
:101670003200f8000100fc000188a900ff3ffc00d7
:101680003200f900ae0120000d0009004f1778006c
:101690004f0778004400f9003600f9004200f900d5
:1016a0000100fc0000400600ff3ffc004200f80083
:1016b0003600f8004400f8008e1f78000e0020006d
:1016c0000d000900be1f78003200f8000100fc0088
:1016d00001a8a900ff3ffc003200f900ae01200084
:1016e0000d0009004f1778004f0778004400f900fb
:1016f0003600f9004200f9000100fc00004006003d
:10170000ff3ffc004200f8003600f8004400f800fb
:101710008e1f78000e0020000d000900be1f78000b
:101720003200f8000100fc000bc8a900ff3ffc00dc
:101730003200f900ae0120000d0009004f177800bb
:101740004f0778004400f9003600f9004200f90024
:101750000100fc0000400600ff3ffc004200f800d2
:101760003600f8004400f8008e1f78000e002000bc
:101770000d000900be1f78003200f8000100fc00d7
:101780000be8a900ff3ffc003200f900ae01200089
:101790000d0009004f1778004f0778004400f9004a
:1017a0003600f9004200f9000100fc00004006008c
:1017b000ff3ffc004200f8003600f8004400f8004b
:1017c0008e1f78000e0020000d000900be1f78005b
:1017d0003200f8000100fc000c08a900ff3ffc00eb
:1017e0003200f900ae0120000d0009004f1778000b
:1017f0004f0778004400f9003600f9004200f90074
:101800000100fc0000400600c0d2bf00bf52e30050
:1018100007003200c072ec00c0d2bf000080fb00a5
:10182000414e210060c07800c3f2b70001003700cc
:10183000c3f2ef0000000600000006003008800040
:10184000109588004008800020958800eeff070072
:10185000c0ccb300c352b50006003900e0cfb300de
:10186000c352b5000100390001003700c472ef0017
:1018700050043700c3f2ae0028003700c472ef00f6
:10188000b0c8b300c352e30005003a00c3d2bf00a2
:10189000c4f2b700c5f2ef00c6f2ef001e00370039
:1018a000b0c9b300c352e30005003a00c3d2bf0081
:1018b000c4f2b700c7f2ef00c8f2ef00160037001d
:1018c000b0cab300c352e30005003a00c3d2bf0060
:1018d000c4f2b700c9f2ef00caf2ef000e00370001
:1018e000b0cbb300c352e30005003a00c3d2bf003f
:1018f000c4f2b700cbf2ef00ccf2ef0006003700e5
:10190000b0ccb300c352e30003003a00c3d2bf001f
:10191000c4f2b700cdf2ef0026043700c452e20053
:1019200002003a002304370022043700b0c8b30095
:10193000c452e300f4003a0000e0ef00c552e300b7
:1019400003003a00c3d2bf00c5f2b700ed00370074
:10195000c3d2bf00c6f2b700e0c5b300c552e30072
:1019600023003a00d572ef00d412a900c652e2005b
:1019700002003600c652d40065f2b7006412e200dd
:1019800013003600d5d2a8006212ec00e090880067
:1019900020938000e29080000200e000020032000c
:1019a000110009000280d800009488000094800093
:1019b000129580002395800000004100e0804900de
:1019c0000001be00c2a68800d3a68800060037002a
:1019d000d8b4ef00dab4ef00262cef002068a9009d
:1019e0000068a90015eea900d312a800c4003700b2
:1019f000f0c5b300c552e30023003a00d672ef00f1
:101a0000d432a900c652e20002003600c652d40009
:101a10006ff2b7006e12e20013003600d6d2a800b3
:101a20006c12ec00e090880070938000e2908000df
:101a30000200e00002003200110009000280d8001c
:101a40004094880040948000129580002395800087
:101a500000004100e08049000001be00e2a68800cd
:101a6000f3a6880006003700dcb4ef00deb4ef0018
:101a7000462cef002368a9000368a90015aea90051
:101a8000d312a8009e00370000c6b300c552e30081
:101a900023003a00d772ef00d452a900c652e200e8
:101aa00002003600c652d40079f2b7007812e20084
:101ab00013003600d7d2a8007612ec00e090880020
:101ac000c0938000e29080000200e000020032003b
:101ad000110009000280d800809488008094800062
:101ae000129580002395800000004100e0804900ad
:101af0000001be0002a7880013a788000600370077
:101b0000e0b4ef00e2b4ef00662cef002388a900f8
:101b10000388a900156ea900d312a8007800370029
:101b2000c5d2bf0080407800efcf500003003a00dc
:101b300010cea90014cea90071003700a0c6b300d2
:101b4000c552e30023003a00d572ef00d412a90079
:101b5000c652e20002003600c652d40065f2b70059
:101b60006412e20013003600d5d2a8006212ec0025
:101b7000e090880020938000e29080000200e00066
:101b800002003200110009000280d8000094880091
:101b90000094800012958000239580000000410091
:101ba000e08049000001be00c2a68800d3a68800dc
:101bb00006003700d8b4ef00dab4ef00262cef00af
:101bc0002068a9000068a90015eea900d312a8009a
:101bd0004b003700b0c6b300c552e30023003a0003
:101be000d672ef00d432a900c652e20002003600dd
:101bf000c652d4006ff2b7006e12e2001300360036
:101c0000d6d2a8006c12ec00e0908800709380009f
:101c1000e29080000200e0000200320011000900a2
:101c20000280d80040948800409480001295800083
:101c30002395800000004100e08049000001be00c3
:101c4000e2a68800f3a6880006003700dcb4ef00a7
:101c5000deb4ef00462cef002368a9000368a9005a
:101c600015aea900d312a80025003700c0c6b300e6
:101c7000c552e30022003a00d772ef00d452a90007
:101c8000c652e20002003600c652d40079f2b70014
:101c90007812e20013003600d7d2a8007612ec00ca
:101ca000e0908800c0938000e29080000200e00095
:101cb00002003200110009000280d80080948800e0
:101cc00080948000129580002395800000004100e0
:101cd000e08049000001be0002a7880013a7880029
:101ce00006003700e0b4ef00e2b4ef00662cef002e
:101cf0002388a9000388a900156ea900d312a800a3
:101d0000c5f2ef002b033700b0c9b300c452e300a3
:101d100071023a0000e0ef00c752e30003003a000e
:101d2000c3d2bf00c7f2b7006a023700c3d2bf00f8
:101d3000c8f2b700c852e200df003a00e0c5b300c5
:101d4000c752e3001f003a00d572ef00d412a90079
:101d50006412e20013003600d5d2a8006212ec0033
:101d6000e090880020938000e29080000200e00074
:101d700002003200110009000280d800009488009f
:101d8000009480001295800023958000000041009f
:101d9000e08049000001be00c2a68800d3a68800ea
:101da00006003700d8b4ef00dab4ef00262cef00bd
:101db0002068a9000068a90015eea900d312a800a8
:101dc000bc003700f0c5b300c752e3001f003a0063
:101dd000d672ef00d432a9006e12e2001300360072
:101de000d6d2a8006c12ec00e090880070938000be
:101df000e29080000200e0000200320011000900c1
:101e00000280d800409488004094800012958000a1
:101e10002395800000004100e08049000001be00e1
:101e2000e2a68800f3a6880006003700dcb4ef00c5
:101e3000deb4ef00462cef002368a9000368a90078
:101e400015aea900d312a8009a00370000c6b3004f
:101e5000c752e3001f003a00d772ef00d452a90026
:101e60007812e20013003600d7d2a8007612ec00f8
:101e7000e0908800c0938000e29080000200e000c3
:101e800002003200110009000280d800809488000e
:101e9000809480001295800023958000000041000e
:101ea000e08049000001be0002a7880013a7880057
:101eb00006003700e0b4ef00e2b4ef00662cef005c
:101ec0002388a9000388a900156ea900d312a800d1
:101ed00078003700c7d2bf0080407800efcf5000b5
:101ee00003003a0010cea90014cea90071003700fb
:101ef000a0c6b300c752e30023003a00d572ef003a
:101f0000d412a900c652e20002003600c652d40024
:101f100065f2b7006412e20013003600d5d2a800c3
:101f20006212ec00e090880020938000e290800034
:101f30000200e00002003200110009000280d80017
:101f40000094880000948000129580002395800002
:101f500000004100e08049000001be00c2a68800e8
:101f6000d3a6880006003700d8b4ef00dab4ef003b
:101f7000262cef002068a9000068a90015eea90032
:101f8000d312a8004b003700b0c6b300c752e3001d
:101f900023003a00d672ef00d432a900c652e20004
:101fa00002003600c652d4006ff2b7006e12e20093
:101fb00013003600d6d2a8006c12ec00e090880026
:101fc00070938000e29080000200e0000200320086
:101fd000110009000280d8004094880040948000dd
:101fe000129580002395800000004100e0804900a8
:101ff0000001be00e2a68800f3a6880006003700b4
:10200000dcb4ef00deb4ef00462cef002368a9003b
:102010000368a90015aea900d312a8002500370057
:10202000c0c6b300c752e30022003a00d772ef00e7
:10203000d452a900c652e20002003600c652d400b3
:1020400079f2b7007812e20013003600d7d2a80068
:102050007612ec00e0908800c0938000e29080004f
:102060000200e00002003200110009000280d800e6
:1020700080948800809480001295800023958000d1
:1020800000004100e08049000001be0002a7880076
:1020900013a7880006003700e0b4ef00e2b4ef00b9
:1020a000662cef002388a9000388a900156ea900fb
:1020b000d312a80087013700e0c5b300c752e30080
:1020c0003d003a00c8d2bf000080fb00f0928800bb
:1020d000d572ef002068a90015eea9005232ef007a
:1020e000a0a48000d0908800409280001a12b50011
:1020f0001092880072958000839580001092800075
:1021000043fa0700c8f9070021fa070090948800f5
:10211000909480004212b500a09488000068a90045
:102120002068a800262cef00d512a800e0928000bd
:10213000f29280000200e00002003200110009006b
:102140000280d800e0938800f19280001093800014
:10215000808f50000d003200109380005e12b50099
:1021600001e0af000020ee00109188000093800095
:10217000129180000200e00002003200110009000c
:102180000280d800f0938800010037007e32ef0013
:10219000e0938000129580002395800000004100ac
:1021a000e08049000001be00c2a68800d3a68800d6
:1021b000d312a80046013700f0c5b300c752e300b0
:1021c0003d003a00c8d2bf000080fb004093880069
:1021d000d672ef002368a90015aea9005432ef00b3
:1021e000b0a48000d0908800509280001a12b500f0
:1021f0002092880092958000a39580002092800014
:1022000003fa070088f90700e1f90700b094880095
:10221000b09480004412b500c09488000368a900ff
:102220002368a800462cef00d612a8003093800047
:10223000429380000200e000020032001100090019
:102240000280d80020948800419380006093800031
:10225000808f50000d003200609380006812b5003e
:1022600001e0af000020ee00109188003093800064
:10227000129180000200e00002003200110009000b
:102280000280d80030948800010037008632ef00c9
:10229000209480001295800023958000000041006a
:1022a000e08049000001be00e2a68800f3a6880095
:1022b000d312a8000601370000c6b300c752e300de
:1022c0003d003a00c8d2bf000080fb009093880018
:1022d000d772ef002388a900156ea9005632ef00cf
:1022e000c0a48000d0908800609280001a12b500cf
:1022f00030928800b2958000c395800030928000b3
:10230000c3f9070048f90700a1f90700d094880035
:10231000d09480004612b500e09488000388a9009c
:102320002388a800662cef00d712a80080938000b5
:10233000929380000200e0000200320011000900c8
:102340000280d8006094880091938000b093800050
:10235000808f50000d003200b09380007212b500e3
:1023600001e0af000020ee00109188008093800013
:10237000129180000200e00002003200110009000a
:102380000280d80070948800010037008e32ef0080
:102390006094800012958000239580000000410029
:1023a000e08049000001be0002a7880013a7880052
:1023b000d312a800c6003700c7d2bf008040780003
:1023c000efcf500003003a0010cea90014cea800b1
:1023d000bf003700a0c6b300c752e3003d003a007b
:1023e000c8d2bf000080fb00f0928800d572ef00d9
:1023f0002068a90015eea9005232ef0060a5800008
:10240000d0908800409280001a12b5001092880087
:102410007295800083958000109280007cf90700ff
:1024200001f907005af90700909488009094800001
:102430004212b500a09488000068a9002068a80096
:10244000262cef00d512a800e0928000f2928000c6
:102450000200e00002003200110009000280d800f2
:10246000e0938800f192800010938000808f5000ec
:102470000d003200109380005e12b50001e0af0045
:102480000020ee00109188000093800012918000df
:102490000200e00002003200110009000280d800b2
:1024a000f0938800010037007e32ef00e093800057
:1024b000129580002395800000004100e0804900d3
:1024c0000001be00c2a68800d3a68800d312a800cf
:1024d0007f003700b0c6b300c752e3003d003a00aa
:1024e000c8d2bf000080fb0040938800d672ef0086
:1024f0002368a90015aea9005432ef0070a5800032
:10250000d0908800509280001a12b5002092880066
:1025100092958000a3958000209280003cf90700ee
:10252000c1f807001af90700b0948800b094800041
:102530004412b500c09488000368a9002368a8006d
:10254000462cef00d612a800309380004293800002
:102550000200e00002003200110009000280d800f1
:10256000209488004193800060938000808f500009
:102570000d003200609380006812b50001e0af00ea
:102580000020ee00109188003093800012918000ae
:102590000200e00002003200110009000280d800b1
:1025a00030948800010037008632ef0020948000cc
:1025b000129580002395800000004100e0804900d2
:1025c0000001be00e2a68800f3a68800d312a8008e
:1025d0003f003700c0c6b300c752e3003c003a00da
:1025e000c8d2bf000080fb0090938800d772ef0034
:1025f0002388a900156ea9005632ef0080a580003f
:10260000d0908800609280001a12b5003092880045
:10261000b2958000c395800030928000fcf80700de
:1026200081f80700daf80700d0948800d094800081
:102630004612b500e09488000388a9002388a8000a
:10264000662cef00d712a800809380009293800040
:102650000200e00002003200110009000280d800f0
:102660006094880091938000b0938000808f500028
:102670000d003200b09380007212b50001e0af008f
:102680000020ee001091880080938000129180005d
:102690000200e00002003200110009000280d800b0
:1026a00070948800010037008e32ef006094800043
:1026b000129580002395800000004100e0804900d1
:1026c0000001be0002a7880013a78800d312a8004b
:1026d000c7f2ef00b7003700b0cab300c452e3003e
:1026e00087003a0000e0ef00c952e30003003a001f
:1026f000c3d2bf00c9f2b70080003700c352ec005c
:10270000caf2b700e0c5b300c952e30012003a00b4
:102710000200200003382400cad2bf00bbf8070023
:10272000fef70700709588008195880072958000fb
:102730008395800010928000b5f807003af80700f2
:1027400093f8070090948800909480004212b5009e
:10275000a094880068003700f0c5b300c952e300b8
:1027600012003a000200200003382400cad2bf0041
:10277000a6f80700e9f7070090958800a195880062
:1027800092958000a395800020928000a0f8070019
:1027900025f807007ef80700b0948800b094800008
:1027a0004412b500c09488005300370000c6b3003f
:1027b000c952e30012003a0002002000033824004e
:1027c000cad2bf0091f80700d4f70700b09588007f
:1027d000c1958800b2958000c3958000309280003a
:1027e0008bf8070010f8070069f80700d0948800fc
:1027f000d09480004612b500e09488003e00370077
:10280000a0c6b300c952e30012003a000200200043
:1028100003382400cad2bf007cf80700bff70700c6
:10282000709588008195880072958000839580005e
:102830001092800076f80700fbf7070054f80700b5
:1028400090948800909480004212b500a094880073
:1028500029003700b0c6b300c952e30012003a00a5
:102860000200200003382400cad2bf0067f8070026
:10287000aaf7070090958800a1958800929580009e
:10288000a39580002092800061f80700e6f707001a
:102890003ff80700b0948800b09480004412b5005f
:1028a000c094880014003700c0c6b300c952e300ca
:1028b00011003a000200200003382400cad2bf00f1
:1028c00052f8070095f70700b0958800c195880079
:1028d000b2958000c3958000309280004cf80700cc
:1028e000d1f707002af80700d0948800d094800020
:1028f0004612b500e0948800c9f2ef002d003700c1
:10290000b0cbb300c452e3000a003a0000e0ef008d
:10291000cb52e30003003a00c3d2bf00cbf2b700b2
:1029200003003700c3d2bf00ccf2b700e6030700b4
:1029300020003700b0ccb300c452e30007003a00d7
:1029400000e0ef00cd52e30003003a00c3d2bf0025
:10295000cdf2b700d203070016003700b0cdb300a8
:10296000c452e30007003a0000e0ef00ce52e3005b
:1029700003003a00c3d2bf00cef2b700d003070075
:102980000c003700b0ceb300c452e30009003a0097
:1029900000e0ef00cf52e30003003a00c3d2bf00d3
:1029a000cff2b70003003700c3d2bf00d0f2b700a8
:1029b000c0030700d312af001903070030c0b300f3
:1029c000d252b500fa0231001295800023958000a2
:1029d0005095800061958000800f5100818f5900d3
:1029e000e8023900adf2a800d252e200f3003a004a
:1029f000d5d2bf0080407800e1cf50000d003a00f2
:102a00007a32ef00d412a90020c0b300d5f2b7008b
:102a1000e093800012958000239580000000410023
:102a2000e08049000001be00c2a68800d3a688004d
:102a3000e1003700d5d2bf0080407800e2cf5000df
:102a400059003a00d1938000f0928000808f5000ae
:102a5000160031007a32ec00d2938000020141006e
:102a6000802d210060007900d0908800d2958000f0
:102a7000e3958000d0908000e5f707006af7070033
:102a8000c3f7070030618800e09380001295800052
:102a90002395800000004100e08049000001be0055
:102aa000c2a68800d3a688003e003700d572ef008a
:102ab000f192800010938000808f500006003a0051
:102ac000d8b4ef00dab4ef0010938000d093880000
:102ad000d412a8003300370010938000f1928000d8
:102ae000808f500018003600d552a800f092800068
:102af000d0938800d293800002014100802d2100f4
:102b000060007900d0908800d2958000e395800025
:102b1000d0908000bef7070043f707009cf707003e
:102b200030618800f093800012958000239580002a
:102b300000004100e08049000001be00c2a68800fc
:102b4000d3a6880017003700d572a800f092800045
:102b5000d0938800d293800002014100802d210093
:102b600060007900d0908800d2958000e3958000c5
:102b7000d0908000a6f707002bf7070084f7070026
:102b800030618800f09380001295800023958000ca
:102b900000004100e08049000001be00c2a688009c
:102ba000d3a6880084003700d5d2bf0080407800cb
:102bb000e4cf50001e003a007a32ed00d29380003c
:102bc00002014100802d210060007900d090880032
:102bd000d2958000e3958000d09080008cf70700ac
:102be00011f707006af7070030618800f093800052
:102bf000129580002395800000004100e08049008c
:102c00000001be00c2a68800d3a68800d193800030
:102c100010938000808f500004003a00d572ef00be
:102c2000d8b4ef00dab4ef00d412a8006200370085
:102c3000d5d2bf0080407800e8cf50001e003a0097
:102c40007a32ec00d293800002014100802d2100f5
:102c500060007900d0908800d2958000e3958000d4
:102c6000d09080006af70700eff6070048f70700ea
:102c700030618800f09380001295800023958000d9
:102c800000004100e08049000001be00c2a68800ab
:102c9000d3a68800d193800010938000808f5000cd
:102ca00004003a00d572ef00d8b4ef00dab4ef00b8
:102cb000d412a8004000370000c4b300d552e3008e
:102cc0001a003a0010938000d0938800d2938000bd
:102cd00002014100802d210060007900d090880021
:102ce000d2958000e3958000d090800048f70700df
:102cf000cdf6070026f707003061880000c8b30052
:102d0000d5f2b700009480001295800023958000d2
:102d100000004100e08049000001be00c2a688001a
:102d2000d3a68800d412a9002300370000c8b3003e
:102d3000d552e30020003a007a12e2001600360075
:102d40007a32ed00d293800002014100802d2100f3
:102d500060007900d0908800d2958000e3958000d3
:102d6000d09080002af70700aff6070008f70700a9
:102d700030618800009480001295800023958000c7
:102d800000004100e08049000001be00c2a68800aa
:102d9000d3a6880008003700d572ef00262cef007c
:102da0000021ef002068a9000068a90015eea90025
:102db000d8b4ef00dab4ef00f1013700d2d2bf008f
:102dc00080407800e1cf5000f5003a00d6d2bf0035
:102dd00080407800e1cf50000d003a008232ef00d1
:102de000d432a90020c0b300d6f2b70020948000ee
:102df000129580002395800000004100e08049008a
:102e00000001be00e2a68800f3a68800e3003700b8
:102e1000d6d2bf0080407800e2cf500059003a007f
:102e20001194800040938000808f50001600310084
:102e30008232ec001294800002014100802d2100ba
:102e400060007900d0908800d2958000e3958000e2
:102e5000d0908000eef6070073f60700ccf607006e
:102e600030628800209480001295800023958000b5
:102e700000004100e08049000001be00e2a6880099
:102e8000f3a688003e003700d672ef004193800021
:102e900060938000808f500006003a00d692a80010
:102ea000dcb4ef00deb4ef00609380001094880083
:102eb000d432a8006093800041938000808f50003e
:102ec00018003600d652a800409380001094880065
:102ed0001294800002014100802d210060007900e1
:102ee000d0908800d2958000e3958000d09080003b
:102ef000c7f607004cf60700a5f607003062880009
:102f000030948000129580002395800000004100dd
:102f1000e08049000001be00e2a68800f3a6880018
:102f200017003700d672a8004093800010948800e4
:102f30001294800002014100802d21006000790080
:102f4000d0908800d2958000e3958000d0908000da
:102f5000aff6070034f607008df6070030628800f0
:102f6000309480001295800023958000000041007d
:102f7000e08049000001be00e2a68800f3a68800b8
:102f800086003700d6d2bf0080407800e4cf5000e2
:102f90001f003a008232ed001294800002014100cd
:102fa000802d210060007900d0908800d2958000ab
:102fb000e3958000d090800095f607001af6070090
:102fc00073f607003062880030948000129580000c
:102fd0002395800000004100e08049000001be0010
:102fe000e2a68800f3a68800119480006093800018
:102ff000808f500005003a00d652a900d692a80052
:10300000dcb4ef00deb4ef00d432a8006300370078
:10301000d6d2bf0080407800e8cf50001f003a00b1
:103020008232ec001294800002014100802d2100c8
:1030300060007900d0908800d2958000e3958000f0
:10304000d090800072f60700f7f5070050f60700f1
:1030500030628800309480001295800023958000b3
:1030600000004100e08049000001be00e2a68800a7
:10307000f3a688001194800060938000808f500038
:1030800005003a00d672a900d692a800dcb4ef0081
:10309000deb4ef00d432a8004000370000c4b30013
:1030a000d652e3001a003a00609380001094880022
:1030b0001294800002014100802d210060007900ff
:1030c000d0908800d2958000e3958000d090800059
:1030d0004ff60700d4f507002df607003062880090
:1030e00000c8b300d6f2b70040948000129580006b
:1030f0002395800000004100e08049000001be00ef
:10310000e2a68800f3a68800d432a9002300370085
:1031100000c8b300d652e30020003a008212e20059
:10312000160036008232ed00129480000201410048
:10313000802d210060007900d0908800d295800019
:10314000e3958000d090800031f60700b6f50700c7
:103150000ff60700306288004094800012958000ce
:103160002395800000004100e08049000001be007e
:10317000e2a68800f3a6880008003700d672ef00a8
:10318000462cef001421ef002368a9000368a90072
:1031900015aea900dcb4ef00deb4ef00f800370094
:1031a000d2d2bf0080407800e2cf5000f4003a0055
:1031b000d7d2bf0080407800e1cf50000d003a0028
:1031c0008a32ef00d452a90020c0b300d7f2b70072
:1031d00060948000129580002395800000004100db
:1031e000e08049000001be0002a7880013a7880004
:1031f000e3003700d7d2bf0080407800e2cf500014
:1032000059003a005194800090938000808f5000c4
:10321000160031008a32ec00529480000201410015
:10322000802d210060007900d0908800d295800028
:10323000e3958000d0908000f5f507007af507004f
:10324000d3f50700306388006094800012958000f9
:103250002395800000004100e08049000001be008d
:1032600002a7880013a788003e003700d772ef003e
:1032700091938000b0938000808f500006003a0048
:10328000d792a800e0b4ef00e2b4ef00d452a80057
:10329000b093800050948800b09380009193800098
:1032a000808f500018003600d752a80090938000fd
:1032b000509488005294800002014100802d21002a
:1032c00060007900d0908800d2958000e39580005e
:1032d000d0908000cef5070053f50700acf507004d
:1032e00030638800709480001295800023958000e0
:1032f00000004100e08049000001be0002a78800f4
:1033000013a7880017003700d772a8009093800099
:10331000509488005294800002014100802d2100c9
:1033200060007900d0908800d2958000e3958000fd
:10333000d0908000b6f507003bf5070094f5070034
:10334000306388007094800012958000239580007f
:1033500000004100e08049000001be0002a7880093
:1033600013a7880086003700d7d2bf0080407800be
:10337000e4cf50001f003a008a32ed0052948000e2
:1033800002014100802d210060007900d09088006a
:10339000d2958000e3958000d09080009cf50700d6
:1033a00021f507007af507003063880070948000eb
:1033b000129580002395800000004100e0804900c4
:1033c0000001be0002a7880013a788005194800066
:1033d000b0938000808f500005003a00d752a900ba
:1033e000d792a800e0b4ef00e2b4ef00d452a800f6
:1033f00063003700d7d2bf0080407800e8cf50008c
:103400001f003a008a32ec00529480000201410011
:10341000802d210060007900d0908800d295800036
:10342000e3958000d090800079f50700fef4070056
:1034300057f5070030638800709480001295800073
:103440002395800000004100e08049000001be009b
:1034500002a7880013a7880051948000b0938000d1
:10346000808f500005003a00d772a900d792a800bb
:10347000e0b4ef00e2b4ef00d452a80040003700ff
:1034800000c4b300d752e3001a003a00b0938000a2
:10349000509488005294800002014100802d210048
:1034a00060007900d0908800d2958000e39580007c
:1034b000d090800056f50700dbf4070034f50700d4
:1034c0003063880000c8b300d7f2b7008094800052
:1034d000129580002395800000004100e0804900a3
:1034e0000001be0002a7880013a78800d452a900db
:1034f0002300370000c8b300d752e30020003a0091
:103500008a12e200160036008a32ed0052948000e2
:1035100002014100802d210060007900d0908800d8
:10352000d2958000e3958000d090800038f50700a8
:10353000bdf4070016f50700306388008094800012
:10354000129580002395800000004100e080490032
:103550000001be0002a7880013a7880008003700fa
:10356000d772ef00662cef001821ef002388a90026
:103570000388a900156ea900e0b4ef00e2b4ef00e3
:1035800027000700a5f2ae0008003700a232ef00c6
:10359000a432ef000821ef000621ef000080eb00cd
:1035a000814d210005000900801878000a003700cd
:1035b000a5f2ae0008003700a232ef00a432ef00ff
:1035c0000821ef000621ef000080eb00814d210073
:1035d000050009008018780089f30700d090880062
:1035e000f09480001a12b60070918800f094800068
:1035f000e09088001c32d500709180001c12b5004c
:1036000000958800128eaa00108ea900a412af00a7
:1036100014eea800a412ae0014eea90087f837003b
:10362000d2f2ef00aab2ef00acb2ef00d172ef001d
:10363000d1d2bf000080fb00c200dd00804d210020
:10364000008040001000be000001be0050958000c8
:1036500061958000800f5100818f59000a00310070
:10366000d1d2bf000080fb00c200dd00804d2100f0
:10367000008040001000be005095880061958800d1
:10368000d1d2bf00d2f2b700d172ec00d1d2bf00cc
:1036900080407800e3cf5000e5ff3a00d312a90044
:1036a00000000600e0c5b300c952e30012003a0072
:1036b0000200200003382400cad2bf00d3f4070060
:1036c00016f4070070958800819588007295800037
:1036d0008395800010928000cdf4070052f407001b
:1036e000abf4070090948800909480004212b500db
:1036f000a094880068003700f0c5b300c952e30009
:1037000012003a000200200003382400cad2bf0091
:10371000bef4070001f4070090958800a195880089
:1037200092958000a395800020928000b8f4070055
:103730003df4070096f40700b0948800b094800030
:103740004412b500c09488005300370000c6b3008f
:10375000c952e30012003a0002002000033824009e
:10376000cad2bf00a9f40700ecf30700b0958800a7
:10377000c1958800b2958000c3958000309280008a
:10378000a3f4070028f4070081f40700d094880010
:10379000d09480004612b500e09488003e003700c7
:1037a000a0c6b300c952e30012003a000200200094
:1037b00003382400cad2bf0094f40700d7f30700ef
:1037c00070958800819588007295800083958000af
:1037d000109280008ef4070013f407006cf40700c9
:1037e00090948800909480004212b500a0948800c4
:1037f00029003700b0c6b300c952e30012003a00f6
:103800000200200003382400cad2bf007ff4070062
:10381000c2f3070090958800a195880092958000da
:10382000a39580002092800079f40700fef3070042
:1038300057f40700b0948800b09480004412b5009b
:10384000c094880014003700c0c6b300c952e3001a
:1038500011003a000200200003382400cad2bf0041
:103860006af40700adf30700b0958800c1958800a1
:10387000b2958000c39580003092800064f4070008
:10388000e9f3070042f40700d0948800d094800048
:103890004612b500e0948800c9f2ef00000006006f
:1038a000cd52e20001003a0091010700cdf2ef0095
:1038b00000000600cff2ef00d0f2ef00000006009b
:1038c000cef2ef0000000600cbd2bf0080407800af
:1038d000e1cf500005003a00ccd2bf000080fb00d1
:1038e0004300dd00f09488003a013700cbd2bf00de
:1038f00080407800e7cf50003a003a00ccd2bf00b9
:103900000080fb00c0928800c2928000020141004a
:10391000802d210060007900d092880002002800ec
:10392000f33f2400d092800039f407007bf30700b6
:10393000d0958800e1958800d412ae000c003700c5
:103940001293800002014100802d21006000790067
:10395000d0908800d2958000e3958000d0908000c0
:103960002bf40700b0f3070009f40700306188006a
:10397000d432ae000c003700629380000201410097
:10398000802d210060007900d0908800d2958000c1
:10399000e3958000d09080001df40700a2f307009b
:1039a000fbf3070030628800d452ae000c003700f1
:1039b000b293800002014100802d21006000790057
:1039c000d0908800d2958000e3958000d090800050
:1039d0000ff4070094f30700edf30700306388004d
:1039e000fc003700cbd2bf0080407800efcf500002
:1039f00011003a00cc72ec000200200003382400d1
:103a0000ccd2bf0001f4070044f307007095880092
:103a10008195880070958000909588008095800041
:103a2000a095880070958000b095880080958000f2
:103a3000c0958800e7003700cbd2bf0080407800f7
:103a4000f0cf50000a003a00ccd2bf000080fb004b
:103a500010938800ccd2bf000080fb0060938800e8
:103a6000ccd2bf000080fb00b0938800d9003700a3
:103a7000cbd2bf0080407800f1cf500007003a0061
:103a8000ccd2bf005df2b700e09280003093880096
:103a9000e092800080938800ce003700cbd2bf0038
:103aa00080407800f2cf500007003a00ccd2bf002f
:103ab00061f2b7000093800050938800009380006b
:103ac000a0938800c3003700cbd2bf0080407800ad
:103ad000f3cf500007003a00cc52d40065f2b70093
:103ae000209380007093880020938000c09388000a
:103af000b8003700cbd2bf0080407800f5cf50002f
:103b00005b003a0081928000ccd2bf000080fb00b5
:103b1000810f500055003200cc52e20002003a0002
:103b20004301070047003700ccd2bf008040780037
:103b3000eccf500002003a00970107004100370027
:103b4000ccd2bf0080407800edcf500002003a0098
:103b5000ea0107003b003700ccd2bf00804078006c
:103b6000eecf500002003a003d020700350037005a
:103b7000ccd2bf0080407800efcf500002003a0066
:103b8000900207002f003700ccd2bf0080407800a1
:103b9000f0cf500002003a00e3020700290037008e
:103ba000ccd2bf0080407800f1cf500002003a0034
:103bb0003603070023003700ccd2bf0080407800d6
:103bc000f2cf500002003a00890307001d003700c1
:103bd000ccd2bf0080407800f3cf500002003a0002
:103be000dc03070017003700ccd2bf00804078000c
:103bf000f4cf500002003a002f04070011003700f4
:103c0000ccd2bf0080407800f5cf500002003a00cf
:103c1000820407000b003700ccd2bf008040780040
:103c2000f6cf500002003a00d50407000500370027
:103c3000ccd2bf0080407800f7cf500001003a009e
:103c400028050700ccd2bf000080fb0080928800ce
:103c50005012e2000300320010cea90014cea800da
:103c60000200370010cea90014cea9005900370079
:103c700020c4b300cb52e30013003a00cc52e20060
:103c800004003a007400070010cea90014cea90069
:103c90000c003700510007005012e20003003a0008
:103ca00010cea90014cea9000200370010cea90042
:103cb00014cea8000821ef000621ef00a232ef0089
:103cc000a432ef004300370060c7b300cb52e300db
:103cd00012003a000200200003302400ccd2bf00c2
:103ce0004af307008df207000200200003f02300d2
:103cf0002bf20700309588004195880032958000ae
:103d0000439580007092800041f30700c6f20700df
:103d1000faf20700409288002e00370070c7b30007
:103d2000cb52e30012003a000200200003302400ce
:103d3000ccd2bf0035f3070078f207000200200064
:103d400003f0230016f207003095880041958800a3
:103d50003295800043958000709280002cf307001c
:103d6000b1f20700e5f20700509288001900370011
:103d700080c7b300cb52e30012003a0002002000db
:103d800003302400ccd2bf0020f3070063f2070009
:103d90000200200003f0230001f2070030958800a4
:103da0004195880032958000439580007092800094
:103db00017f307009cf20700d0f20700609288001a
:103dc00004003700b0c7b300cb52e30001003a0053
:103dd00002000700cbf2ef0000000600262cef00e7
:103de000462cef00662cef002068a9002368a9008c
:103df0002388a90015eea90015aea900156ea9002b
:103e0000d572ef00d672ef00d772ef00d472ef00d8
:103e1000d172ef0020c0b300d152e3000a003e008f
:103e2000d1d2bf000080fb00c200dd00804d210028
:103e300000814000f0ff2f00f1ff2f000089be003d
:103e4000d172ec00f3ff3900d2f2ef00aab2ef001a
:103e5000acb2ef0000000600d172ef0020c0b3004a
:103e6000d152e3000a003e00d1d2bf000080fb0027
:103e7000c200dd00804d210000814000f0ff2f00d6
:103e8000f1ff2f000089be00d172ec00f3ff390072
:103e9000d2f2ef00aab2ef00acb2ef00262cef0096
:103ea000462cef00662cef002068a9002368a900cb
:103eb0002388a90011eea90015eea90011aea900f2
:103ec00015aea900116ea900156ea900d572ef00fc
:103ed000d672ef00d772ef00d472ef000400070033
:103ee0004832ef004a32ef004c32ef00500037000a
:103ef000f0072000c0928800c292800002014100b9
:103f0000802d210060007900d092880002002800f6
:103f1000f33f2400d0928000bdf20700fff10700bc
:103f2000d0958800e1958800a0c0b3005df2b7008d
:103f300040c1b30061f2b700600720001093880011
:103f4000a0c0b30065f2b7004832ef0060ec230078
:103f500080958800ae32ef0000042000f0948800c5
:103f6000e092800030938800009380005093880096
:103f700010938000609388002093800070938800e5
:103f80004a32ef00709580009095880080958000ff
:103f9000a0958800e09280008093880000938000c4
:103fa000a093880010938000b09388002093800035
:103fb000c09388004c32ef0070958000b095880067
:103fc00080958000c09588000000060010c0b300f6
:103fd000d1f2b700f0c7b300d152e30010003e00a9
:103fe000d1d2bf0089f2070035f107000001be0001
:103ff00090c22500512324000bf2070064f2070051
:10400000112d2100914078008180fb0081804000cb
:10401000822d210080307900d172ec00edff390053
:10402000f01f2000b09e8800d832ef00000006008c
:1040300080fa2d0000a4880060312d0010a48800b3
:1040400080732c0020a4880060c02b0030a488005e
:1040500040172b0040a48800a0772a0050a48800b5
:10406000f0e0290060a48800c052290070a48800f4
:1040700080cc280080a48800d04d280090a488001f
:1040800030d62700a0a4880050652700b0a488007f
:10409000d0fa2600c0a4880040962600d0a488004c
:1040a00050372600e0a48800c0dd2500f0a4880079
:1040b0003089250000a588006039250010a58800fa
:1040c00000ee240020a58800f0a6240030a588007a
:1040d000d063240040a588007024240050a58800e7
:1040e000b0e8230060a5880040b0230070a58800d8
:1040f000f07a230080a58800b048230090a58800ae
:1041000030192300a0a5880070ec2200b0a588001b
:1041100020c22200c0a58800409a2200d0a58800b5
:1041200090742200e0a5880000512200f0a58800cc
:10413000702f220000a68800d00f220010a6880051
:10414000e0f1210020a68800b0d5210030a688002b
:1041500010bb210040a68800e0a1210050a68800e5
:10416000308a210060a68800c073210070a68800f4
:10417000a05e210080a68800b04a210090a6880099
:10418000d0372100a0a6880010262100b0a6880004
:10419000d8b3ef000000060080fa2d0000a48800cc
:1041a000801a2d0010a48800506c2c0020a48800d8
:1041b00040a52b0030a48800d02d2b0040a48800ff
:1041c000a07a2a0050a4880050ef290060a488003b
:1041d0000050290070a48800b0ba280080a488008c
:1041e0002061280090a48800e0c12700a0a48800d6
:1041f00040722700b0a48800d0fa2600c0a488002e
:10420000d08a2600d0a48800b0332600e0a488001d
:1042100030d02500f0a488007094250000a5880007
:10422000e03a250010a5880030f5240020a588007c
:1042300090a5240030a58800f05a240040a58800ed
:10424000202e240050a5880080de230060a5880071
:10425000b0b6230070a58800f07a230080a58800fe
:10426000f042230090a5880070172300a0a58800c5
:10427000a0e52200b0a58800d0c72200c0a5880014
:10428000009b2200d0a5880020782200e0a58800ad
:1042900050502200f0a58800002b220000a68800c4
:1042a000a014220010a68800d0ec210020a68800cf
:1042b000e0d8210030a6880010bb210040a688006d
:1042c000109f210050a688004089210060a6880028
:1042d0006070210070a688007061210080a68800af
:1042e000104b210090a68800a0392100a0a68800cc
:1042f000c0252100b0a6880000000600d0122e00c4
:1043000000a4880060312d0010a48800f05d2c000e
:1043100020a4880090b92b0030a48800a0fd2a00ba
:1043200040a48800f08c2a0050a48800d0e3290023
:1043300060a488004060290070a48800f0c92800ab
:1043400080a48800003d280090a4880070e8270021
:10435000a0a4880020522700b0a4880000072700ee
:10436000c0a4880040962600d0a48800902c260087
:10437000e0a4880050da2500f0a48800607c2500c5
:1043800000a588000044250010a5880070ef2400d7
:1043900020a58800b0ad240030a5880080622400ec
:1043a00040a58800101c240050a58800d0f12300ef
:1043b00060a58800a0a6230070a5880010812300b6
:1043c00080a58800b048230090a58800d013230062
:1043d000a0a58800c0ea2200b0a58800c0bb2200ca
:1043e000c0a58800909f2200d0a5880050752200ab
:1043f000e0a5880060542200f0a58800d02e22009d
:1044000000a68800900b220010a6880070f62100fc
:1044100020a68800e0d0210030a6880010be210030
:1044200040a68800e0a1210050a6880080872100d6
:1044300060a68800f072210070a68800705b2100e1
:1044400080a68800504d210090a6880030382100b9
:10445000a0a68800c0272100b0a6880000000600a2
:1044600090022e0000a4880060482d0010a488004f
:1044700080732c0020a4880000ac2b0030a488009e
:10448000d0102b0040a48800705f2a0050a4880040
:1044900010f5290060a488007055290070a48800d8
:1044a00040d9280080a48800604b280090a4880090
:1044b00060c62700a0a4880090762700b0a48800da
:1044c000b0e82600c0a48800c0a12600d0a48800bf
:1044d00050372600e0a4880090d32500f0a488007f
:1044e000f085250000a58800502d250010a5880026
:1044f00010f8240020a5880040a8240030a58800da
:10450000306a240040a588004023240050a588007c
:10451000c0e0230060a58800d0b8230070a5880003
:10452000e071230080a58800704e230090a58800cc
:1045300030192300a0a5880050e72200b0a588000c
:1045400090c02200c0a5880030942200d0a5880029
:10455000a0792200e0a58800b0512200f0a58800d3
:10456000a032220000a68800300f220010a688008a
:10457000f0ed210020a6880000da210030a6880096
:1045800080b6210040a68800c0a4210050a6880063
:10459000308a210060a688004071210070a6880042
:1045a000d05d210080a68800a047210090a6880049
:1045b000603a2100a0a6880060262100b0a68800ed
:1045c00000000600001b2e0000a4880000392d000a
:1045d00010a4880040892c0020a4880060c02b0013
:1045e00030a4880000042b0040a4880090712a00a9
:1045f00050a4880020ca290060a48800b065290062
:1046000070a4880010cf280080a48800e0592800fa
:1046100090a48800f0d32700a0a48800605627004b
:10462000b0a48800100b2700c0a4880020852600b5
:10463000d0a4880030422600e0a48800c0dd250018
:10464000f0a48800907f250000a588005036250042
:1046500010a58800a0e2240020a5880070b02400e6
:1046600030a588001065240040a58800802a240019
:1046700050a5880080e7230060a58800c0a823001b
:1046800070a588001083230080a5880020402300a7
:1046900090a58800a01e2300a0a5880070ec220031
:1046a000b0a5880050bd2200c0a58800c098220097
:1046b000d0a58800e06e2200e0a58800c055220049
:1046c000f0a588002030220000a68800d012220029
:1046d00010a6880050f1210020a68800f0d121000a
:1046e00030a6880020bf210040a68800a09d2100a0
:1046f00050a68800e08c210060a68800c0732100cd
:1047000070a68800405c210080a68800f049210046
:1047100090a6880000352100a0a6880070282100fe
:10472000b0a688000000060040de2d0000a488002e
:1047300010502d0010a48800c07a2c0020a48800fe
:10474000d0d42b0030a4880040172b0040a4880050
:1047500080652a0050a4880030db290060a488000e
:10476000303d290070a4880070de280080a48800f5
:104770003050280090a48800a0e12700a0a4880061
:1047800030632700b0a48800b0ec2600c0a48800e5
:1047900090a52600d0a4880030272600e0a4880039
:1047a00000e82500f0a488003089250000a58800d5
:1047b0005030250010a5880030eb240020a588008b
:1047c000309c240030a58800c06c240040a58800df
:1047d000b025240050a5880060ee230060a5880065
:1047e00020af230070a58800e073230080a5880017
:1047f0006050230090a5880020112300a0a5880008
:1048000090f12200b0a5880020c22200c0a5880037
:10481000b0952200d0a5880020732200e0a5880072
:10482000a04b2200f0a58800f033220000a68800eb
:104830006010220010a68800c0f4210020a6880085
:1048400020d5210030a6880080b7210040a688002e
:10485000c0a5210050a688002086210060a68800ff
:104860005076210070a68800a05e210080a68800f6
:104870007048210090a6880020372100a0a688005b
:1048800060232100b0a688000000060070f62d000d
:1048900000a48800c0162d0010a4880080902c0071
:1048a00020a4880030c72b0030a48800902a2b0059
:1048b00040a48800a0772a0050a48800d0cf290007
:1048c00060a48800504d290070a4880030b82800ea
:1048d00080a48800b05e280090a4880080d82700bb
:1048e000a0a4880010702700b0a48800c0f826009b
:1048f000c0a48800f0882600d0a48800d0452600f7
:10490000e0a4880080ce2500f0a48800d092250085
:1049100000a588006039250010a5880070e52400f6
:1049200020a5880040a4240030a58800a0592400b8
:1049300040a58800f02c240050a58800d0e9230071
:1049400060a58800a0b5230070a58800f079230039
:1049500080a588000042230090a5880070202300d5
:10496000a0a58800d0e42200b0a5880000c72200de
:10497000c0a58800409a2200d0a58800507022006f
:10498000e0a58800b04f2200f0a58800602a220030
:1049900000a688000014220010a6880070f22100f2
:1049a00020a6880060d8210030a6880080ba2100a7
:1049b00040a68800909e210050a68800d08d21003e
:1049c00060a68800f06f210070a6880010612100a9
:1049d00080a68800b04a210090a68800b03521004a
:1049e000a0a6880060252100b0a68800000006006f
:1049f00050e62d0000a48800902d2d0010a4880002
:104a0000605a2c0020a48800b0db2b0030a4880062
:104a1000b01d2b0040a48800e0892a0050a4880023
:104a2000f0e0290060a488009042290070a488006a
:104a300060c7280080a48800a03a280090a48800bd
:104a400030e62700a0a4880080672700b0a4880073
:104a5000f0042700c0a4880050942600d0a4880049
:104a6000c02a2600e0a4880060eb2500f0a488009e
:104a7000d07a250000a588008042250010a5880076
:104a800000ee240020a58800d09e240030a58800d8
:104a90004061240040a58800e01a240050a5880049
:104aa000a0f0230060a5880050b1230070a5880005
:104ab0000080230080a58800c047230090a58800bf
:104ac000f0122300a0a5880040f32200b0a58800c2
:104ad000f0ba2200c0a58800d09e2200d0a5880090
:104ae00090742200e0a58800004d2200f0a5880007
:104af000302e220000a68800000b220010a688009d
:104b0000e0f5210020a6880030d6210030a68800dc
:104b100090bd210040a6880070a1210050a6880009
:104b20000087210060a688003077210070a68800e9
:104b3000105b210080a68800f04c210090a6880020
:104b4000d0372100a0a6880010242100b0a688003c
:104b50000000060080fe2d0000a48800501e2d00dd
:104b600010a48800f06f2c0020a48800a0a82b00bf
:104b700030a4880010312b0040a48800b07d2a00aa
:104b800050a4880030f2290060a48800c052290097
:104b900070a4880040bd280080a488000049280037
:104ba00090a4880020c42700a0a488006074270077
:104bb000b0a48800d0fc2600c0a48800d09f2600a6
:104bc000d0a4880080352600e0a48800e0d125002c
:104bd000f0a488001096250000a58800d02b2500a1
:104be00010a58800a0f6240020a58800f0a62400c7
:104bf00030a58800305c240040a5880010222400e5
:104c000050a58800a0df230060a58800c0b723005e
:104c100070a58800f07b230080a58800704d2300dc
:104c200090a5880050182300a0a5880080e62200e7
:104c3000b0a58800a0c82200c0a5880070932200fb
:104c4000d0a58800e0782200e0a58800005122006d
:104c5000f0a58800a02b220000a68800900e22005c
:104c600010a6880060ed210020a6880070d92100e0
:104c700030a6880090bb210040a6880050a42100e7
:104c800050a68800b089210060a68800d07021005d
:104c900070a68800e061210080a6880040472100be
:104ca00090a68800003a2100a0a6880010262100c6
:104cb000b0a6880000000600f0162e0000a48800b0
:104cc00030352d0010a4880090612c0020a48800ad
:104cd000f0bc2b0030a48800d0002b0040a488003a
:104ce000f08f2a0050a48800b0e6290060a4880054
:104cf0000063290070a4880080cc280080a488006c
:104d0000603f280090a48800b0d12700a0a48800ac
:104d100040542700b0a4880000092700c0a48800e0
:104d200020982600d0a4880060402600e0a48800d7
:104d300000dc2500f0a48800007e250000a5880086
:104d40009045250010a5880030e1240020a58800aa
:104d500010af240030a58800d063240040a588004f
:104d6000401d240050a5880060e6230060a588004f
:104d7000b0a7230070a588001082230080a58800ba
:104d8000a049230090a58800c01d2300a0a588008d
:104d900090eb2200b0a5880090bc2200c0a588003e
:104da00050a02200d0a58800306e2200e0a5880027
:104db00010552200f0a58800702f220000a6880060
:104dc000300c220010a68800c0f0210020a6880028
:104dd00060d1210030a6880090be210040a6880046
:104de00060a2210050a68800708c210060a6880077
:104df0005073210070a68800d05b210080a6880037
:104e0000b04d210090a68800a0342100a0a6880003
:104e100020282100b0a688000000060040da2d00fe
:104e200000a48800304c2d0010a4880020772c00ae
:104e300020a4880060af2b0030a4880000142b0051
:104e400040a4880070622a0050a48800f0f729006e
:104e500060a488002058290070a48800d0db2800b6
:104e600080a48800d04d280090a48800a0c8270006
:104e7000a0a4880010612700b0a48800b0ea260032
:104e8000c0a48800b0a32600d0a488002039260042
:104e9000e0a4880040e62500f0a488009087250063
:104ea00000a58800d02e250010a5880080f92400d8
:104eb00020a58800d09a240030a58800806b2400ab
:104ec00040a588007024240050a58800e0e123005c
:104ed00060a5880010ae230070a58800e072230052
:104ee00080a58800604f230090a58800201a230029
:104ef000a0a58800b0f02200b0a5880050c1220013
:104f0000c0a58800f0942200d0a58800507a220025
:104f1000e0a58800f04a2200f0a588005033220066
:104f200000a68800d00f220010a6880080ee210085
:104f300020a68800a0d4210030a6880000b7210058
:104f400040a6880040a5210050a68800a08a210024
:104f500060a68800e075210070a68800405e2100f0
:104f600080a688000048210090a68800b03a210061
:104f7000a0a6880010232100b0a68800000006002b
:104f8000101f2e0000a48800f0122d0010a488002d
:104f9000e08c2c0020a48800c0c32b0030a4880023
:104fa00030072b0040a4880090742a0050a4880089
:104fb00000cd290060a488007068290070a48800d2
:104fc000a0d1280080a48800405c280090a488001c
:104fd00030d62700a0a4880080582700b0a48800fd
:104fe000c0f62600c0a4880000872600d0a4880050
:104ff00000442600e0a4880070df2500f0a48800ab
:105000004091250000a58800d037250010a5880014
:1050100010e4240020a58800c0b1240030a5880039
:105020006058240040a58800b02b240050a58800bb
:10503000b0e8230060a58800d0a9230070a58800ef
:10504000f078230080a588001041230090a58800f7
:10505000901f2300a0a5880040ed2200b0a5880085
:1050600030c62200c0a5880080992200d0a5880003
:10507000906f2200e0a5880070562200f0a58800fd
:10508000c029220000a688006013220010a6880014
:10509000e0f1210020a6880070d2210030a688000f
:1050a00000ba210040a68800109e210050a688006a
:1050b000508d210060a688003074210070a6880001
:1050c000a060210080a68800504a210090a6880098
:1050d00060352100a0a68800c0282100b0a6880065
:1050e0000000060040e22d0000a48800f0532d00cf
:1050f00010a48800d0562c0020a4880040d82b0093
:1051000030a48800701a2b0040a4880080682a0010
:1051100050a4880010de290060a48800e03f290028
:1051200070a4880000e1280080a48800a052280014
:1051300090a48800e0e32700a0a488005065270021
:10514000b0a48800b0ee2600c0a4880070922600ab
:10515000d0a48800f0282600e0a48800b0e925004b
:10516000f0a48800c08a250000a58800f040250032
:1051700010a5880090ec240020a58800809d2400c4
:1051800030a58800106e240040a58800b0192400c6
:1051900050a5880080ef230060a5880040b0230060
:1051a00070a58800e074230080a58800c046230015
:1051b00090a5880010122300a0a5880060f22200ac
:1051c000b0a58800f0c22200c0a58800109e220071
:1051d000d0a58800e0732200e0a58800504c220092
:1051e000f0a588009034220000a68800600a220002
:1051f00010a6880050f5210020a68800b0d5210017
:1052000030a6880000b8210040a68800f0a0210048
:1052100050a688009086210060a68800c0762100f4
:1052200070a68800005f210080a68800904c2100b5
:1052300090a6880080372100a0a68800b023210016
:08524000b0a688000000060082
:020000040000fa
:105248001a12000014000000800000002e12000056
:105258007400000080000000a21200001c00000082
:1052680080000000be1200001a000000800000004c
:10527800d81200000002000080000000d8140000ce
:105288000c00000080000000e41400000a02000086
:0852980080000000000000008e
:00000001FF
